:020000040000FA
:020000003B289B
:08000800A92A08208600080067
:10001000BD0000308A003D08820740347934243422
:1000200030341934123402347834003410346334E8
:100030007F3086000800BD0000308A0038303D0265
:100040008207ED345634EE346234EF345F34F034EA
:100050004E34F1343034F2340534F234CD34F334E8
:100060008B34F4343E34F434E734F5348634F634E7
:100070001D34F634AB3403138312850107309F001F
:100080008316303085008601803081000C10831289
:100090008B12013090000B178B170F3085006822F0
:1000A0007F20AC010530BB00FA30BA002B21BA0B1F
:1000B0005628BB0B542820308400831626309B0022
:1000C000831283161C141A089B0A83128000840A68
:1000D00024300402031D6128A401A501A601A80182
:1000E000A701AC0174209C288B128330810024303E
:1000F000A900D730AA003C30AB008B160800203096
:1001000084000030B1009630B2005322003E031943
:10011000952880002E3C0319852830300002031CEE
:10012000932830308002840A852808000A3431344C
:100130002E343034363400342B212718DE28A7180B
:10014000FE28A5080319A628A50B9C28182005142D
:10015000051EFB21051A072283161F308600831215
:10016000061C9721861CB021061DC921861DE2218F
:10017000061E4821831686018312AB08031D9C28A6
:100180008B120F3085000530BC006D22A122A12208
:10019000A122BC0BC5287322732283160616831274
:1001A0008B156300061AD02832309122061ED628FD
:1001B000323091228316061283125B28051AE22838
:1001C0007922FD28281C9C288B1223080520851ED7
:1001D000F3280530BC0068221E3091226822A1223B
:1001E000BC0BEB28FD280230BC000130B1000E3002
:1001F000B2001222A322BC0BF5285B28051A9C280A
:100200008B127922A1227922A701AC0174202B2123
:10021000AB080319C028051A07295B28C03423340A
:100220008034083423340434253404342734183417
:10023000253404342334043480340C34233404341B
:10024000253404342734043425340434233404346A
:100250002534203400342C18452918200514851124
:10026000200805208F22182085150511210805205A
:100270008F22182005158510220805208F221820AE
:1002800085140510230805208F2218200514080066
:100290002408031D4D293330A400A40B9629261CE5
:1002A0005929A301A201A101A0018230A500742057
:1002B00096298B122308031D68292208031D68292B
:1002C0002108031D68292008031D6829A7148E2909
:1002D00020308400831626309B00831283161C1462
:1002E0001A088312000203198529000883169A0050
:1002F0001C1555309D00AA309D009C149C187E2929
:1003000083128C1383161C11831283169B0A83128B
:10031000840A24300402031D6E29271483308100CF
:100320002430A900D730AA00AC018B16080024089D
:10033000031D9C293330A400A40BAF292618A6293D
:10034000A30A0A3023020318A301AC290130A30237
:100350000318AC290930A3008230A50074200800DE
:100360002408031DB5293330A400A40BC82926187E
:10037000BF29A20A063022020318A201C5290130B2
:10038000A2020318C5290530A2008230A5007420FE
:1003900008002408031DCE293330A400A40BE12952
:1003A0002618D829A10A0A3021020318A101DE2942
:1003B0000130A1020318DE290930A1008230A50016
:1003C000742008002408031DE7293330A400A40B7F
:1003D000FA292618F129A00A0A3020020318A001E0
:1003E000F7290130A0020318F7290930A000823054
:1003F000A500742008002618062A2408031D022AD6
:100400003330A400A40B062A261474200800261CEE
:10041000112A2408031D0E2A3330A400A40B112A2C
:10042000261008000130B0005322AD002D0803193A
:100430004A2A5322AE0080302D0203193C2AC030D4
:100440002D02031D262A2E08AF00472AC1302D0297
:10045000031D312A3108B3003208B4002E08B00061
:10046000472A03102D0D1B20B50003142D0D1B2052
:10047000B60083160C1483122F08BB0001309122A2
:10048000BB0B3E2AAE0B3C2A83160C108312051AB6
:10049000142A522AB00B4D2A522A3308B1003408CC
:1004A000B200142A08005822B20A0319B10A08003F
:1004B00031088A0032088200F630B500AB30B60051
:1004C00064307D2AF330B5008B30B60064307D2A6D
:1004D00062221E3091225C220800ED30B5005630B9
:1004E000B60064307D2AED30B5005630B600FA30E3
:1004F0007D2A6D229D227322080083160C1483121C
:10050000912283160C10831208000530B7000000FA
:1005100000000000B70B892A08003C30862AB8305A
:10052000862AB9000A30B800952A962A00008D2242
:10053000B80B962AB90B922A08006430912AC83069
:10054000912AFA30912A0A30BA009D22BA0BA52AC4
:100550000800F0000308F10083120B19B42A0C18EC
:10056000D92A0B18E12AE32A0B11833081000130CC
:10057000AA020319BF2A0318E32AA902E32AA90839
:10058000031DD12A2430A900D730AA00AC012718B6
:10059000CD2AA718CF2AAB03E32AE822E32A1023A7
:1005A000E32A27080319E32A1C302902031C2C1410
:1005B000E32A0C1035088F0036088E00803086063E
:1005C000E32A0B108B1171088300F00E700E0900E6
:1005D000230BF62A2208031DF62A2108031DF62AFA
:1005E0002008031DF62AA30328140F2B2308031940
:1005F000FB2AA3030F2B0930A30022080319022BA7
:10060000A2030F2B0530A20021080319092BA10317
:100610000F2B0930A100200803190F2BA00308009D
:10062000A30A0A302302031C282BA301A20A0630C6
:100630002202031C282BA201A10A0A302102031C5A
:10064000282BA101A00A0A302002031C282BA0019C
:020650000800A0
:02400E00023F6F
:1042000043006F0070007900720069006700680069
:1042100074002000280043002900200032003000F4
:10422000310030002D003200300031003900200014
:104230006200790020004D002E00590061006D00E1
:1042400061006D006F0074006F00FF00000000004F
:04425000000000006A
:00000001FF
